 pwm

 Timestamp is 4da2a53f (Mon Apr 11 18:52:47 2011)

 Preferred load address is 10000000

 Start         Length     Name                   Class
 0001:00000000 000008a8H .rdata                  CODE
 0001:000008a8 00000020H .rdata$debug            CODE
 0001:000008c8 00001d60H .text                   CODE
 0001:00002628 00000004H .xdata                  CODE
 0001:0000262c 0000003cH .idata$2                CODE
 0001:00002668 00000014H .idata$3                CODE
 0001:0000267c 0000006cH .idata$4                CODE
 0001:000026e8 00000060H .idata$6                CODE
 0001:00002750 000000ecH .edata                  CODE
 0002:00000000 0000006cH .idata$5                DATA
 0002:00000070 0000044cH .data                   DATA
 0003:00000000 000000f0H .pdata                  DATA

  Address         Publics by Value              Rva+Base       Lib:Object

 0000:00000000       ___safe_se_handler_table   00000000     <absolute>
 0000:00000000       ___safe_se_handler_count   00000000     <absolute>
 0001:0000001c       ??_C@_1BK@KMGMHKOK@?$AA?$CL?$AA?$CL?$AAP?$AAW?$AAM?$AA_?$AAI?$AAn?$AAi?$AAt?$AA?$AN?$AA?6?$AA?$AA@ 1000101c     pwm_mx25_topaz_v1:pwmmdd.obj
 0001:00000038       ??_C@_1BO@IHNIPGBF@?$AA?9?$AA?9?$AAP?$AAW?$AAM?$AA_?$AAD?$AAe?$AAi?$AAn?$AAi?$AAt?$AA?$AN?$AA?6?$AA?$AA@ 10001038     pwm_mx25_topaz_v1:pwmmdd.obj
 0001:00000058       ??_C@_1BO@LCGLCGL@?$AA?$CL?$AA?$CL?$AAP?$AAW?$AAM?$AA_?$AAD?$AAe?$AAi?$AAn?$AAi?$AAt?$AA?$AN?$AA?6?$AA?$AA@ 10001058     pwm_mx25_topaz_v1:pwmmdd.obj
 0001:00000078       ??_C@_1BK@MJCDENDC@?$AA?9?$AA?9?$AAP?$AAW?$AAM?$AA_?$AAO?$AAp?$AAe?$AAn?$AA?$AN?$AA?6?$AA?$AA@ 10001078     pwm_mx25_topaz_v1:pwmmdd.obj
 0001:00000094       ??_C@_1M@FBHMHEOP@?$AAP?$AAW?$AAM?$AA4?$AA?3?$AA?$AA@ 10001094     pwm_mx25_topaz_v1:pwmmdd.obj
 0001:000000a0       ??_C@_1M@EMHJEEFH@?$AAP?$AAW?$AAM?$AA3?$AA?3?$AA?$AA@ 100010a0     pwm_mx25_topaz_v1:pwmmdd.obj
 0001:000000ac       ??_C@_1M@IHCFJHPC@?$AAP?$AAW?$AAM?$AA2?$AA?3?$AA?$AA@ 100010ac     pwm_mx25_topaz_v1:pwmmdd.obj
 0001:000000b8       ??_C@_1M@BLBOFFM@?$AAP?$AAW?$AAM?$AA1?$AA?3?$AA?$AA@ 100010b8     pwm_mx25_topaz_v1:pwmmdd.obj
 0001:000000c4       ??_C@_1BK@EGMAMCND@?$AA?$CL?$AA?$CL?$AAP?$AAW?$AAM?$AA_?$AAO?$AAp?$AAe?$AAn?$AA?$AN?$AA?6?$AA?$AA@ 100010c4     pwm_mx25_topaz_v1:pwmmdd.obj
 0001:000000e0       ??_C@_1BM@EHKJFHBN@?$AA?9?$AA?9?$AAP?$AAW?$AAM?$AA_?$AAC?$AAl?$AAo?$AAs?$AAe?$AA?$AN?$AA?6?$AA?$AA@ 100010e0     pwm_mx25_topaz_v1:pwmmdd.obj
 0001:000000fc       ??_C@_1BM@HNMLIEOC@?$AA?$CL?$AA?$CL?$AAP?$AAW?$AAM?$AA_?$AAC?$AAl?$AAo?$AAs?$AAe?$AA?$AN?$AA?6?$AA?$AA@ 100010fc     pwm_mx25_topaz_v1:pwmmdd.obj
 0001:00000118       ??_C@_1CE@NANENLHD@?$AA?9?$AA?9?$AAP?$AAW?$AAM?$AA_?$AAP?$AAo?$AAw?$AAe?$AAr?$AAD?$AAo?$AAw?$AAn?$AA?$AN?$AA?6?$AA?$AA@ 10001118     pwm_mx25_topaz_v1:pwmmdd.obj
 0001:0000013c       ??_C@_1CE@MCBJMKDL@?$AA?$CL?$AA?$CL?$AAP?$AAW?$AAM?$AA_?$AAP?$AAo?$AAw?$AAe?$AAr?$AAD?$AAo?$AAw?$AAn?$AA?$AN?$AA?6?$AA?$AA@ 1000113c     pwm_mx25_topaz_v1:pwmmdd.obj
 0001:00000160       ??_C@_1CA@MOKADFEP@?$AA?9?$AA?9?$AAP?$AAW?$AAM?$AA_?$AAP?$AAo?$AAw?$AAe?$AAr?$AAU?$AAp?$AA?$AN?$AA?6?$AA?$AA@ 10001160     pwm_mx25_topaz_v1:pwmmdd.obj
 0001:00000180       ??_C@_1CA@OKNGIEA@?$AA?$CL?$AA?$CL?$AAP?$AAW?$AAM?$AA_?$AAP?$AAo?$AAw?$AAe?$AAr?$AAU?$AAp?$AA?$AN?$AA?6?$AA?$AA@ 10001180     pwm_mx25_topaz_v1:pwmmdd.obj
 0001:000001a0       ??_C@_1BK@BEPLCHFL@?$AA?9?$AA?9?$AAP?$AAW?$AAM?$AA_?$AAR?$AAe?$AAa?$AAd?$AA?$AN?$AA?6?$AA?$AA@ 100011a0     pwm_mx25_topaz_v1:pwmmdd.obj
 0001:000001bc       ??_C@_1BK@JLBIKILK@?$AA?$CL?$AA?$CL?$AAP?$AAW?$AAM?$AA_?$AAR?$AAe?$AAa?$AAd?$AA?$AN?$AA?6?$AA?$AA@ 100011bc     pwm_mx25_topaz_v1:pwmmdd.obj
 0001:000001d8       ??_C@_1BM@NFHHPCHB@?$AA?9?$AA?9?$AAP?$AAW?$AAM?$AA_?$AAW?$AAr?$AAi?$AAt?$AAe?$AA?$AN?$AA?6?$AA?$AA@ 100011d8     pwm_mx25_topaz_v1:pwmmdd.obj
 0001:000001f4       ??_C@_1BM@OPBFCBIO@?$AA?$CL?$AA?$CL?$AAP?$AAW?$AAM?$AA_?$AAW?$AAr?$AAi?$AAt?$AAe?$AA?$AN?$AA?6?$AA?$AA@ 100011f4     pwm_mx25_topaz_v1:pwmmdd.obj
 0001:00000210       ??_C@_1EI@OHOBDPNN@?$AAP?$AAW?$AAM?$AA_?$AAI?$AAO?$AAC?$AAo?$AAn?$AAt?$AAr?$AAo?$AAl?$AA?3?$AA?5?$AAN?$AAo?$AA?5?$AAm?$AAa?$AAt?$AAc?$AAh?$AAi?$AAn?$AAg?$AA?5?$AAI?$AAO?$AAC?$AAT?$AAL@ 10001210     pwm_mx25_topaz_v1:pwmmdd.obj
 0001:00000258       ??_C@_1HG@CLLFEGEM@?$AAD?$AAU?$AAM?$AA_?$AAI?$AAO?$AAC?$AAo?$AAn?$AAt?$AAr?$AAo?$AAl?$AA?3?$AA?5?$AAI?$AAO?$AAC?$AAT?$AAL?$AA_?$AAP?$AAO?$AAW?$AAE?$AAR?$AA_?$AAS?$AAE?$AAT?$AA?3?$AA?5@ 10001258     pwm_mx25_topaz_v1:pwmmdd.obj
 0001:000002d0       ??_C@_1EM@PBEHOOGP@?$AAP?$AAW?$AAM?$AA_?$AAI?$AAO?$AAC?$AAo?$AAn?$AAt?$AAr?$AAo?$AAl?$AA?3?$AA?5?$AAP?$AAW?$AAM?$AA_?$AAI?$AAO?$AAC?$AAT?$AAL?$AA_?$AAG?$AAE?$AAT?$AAC?$AAL?$AAK?$AAF@ 100012d0     pwm_mx25_topaz_v1:pwmmdd.obj
 0001:00000320       ??_C@_1EC@KALNMFCG@?$AAP?$AAW?$AAM?$AA_?$AAI?$AAO?$AAC?$AAo?$AAn?$AAt?$AAr?$AAo?$AAl?$AA?3?$AA?5?$AAP?$AAW?$AAM?$AA_?$AAI?$AAO?$AAC?$AAT?$AAL?$AA_?$AAR?$AAE?$AAS?$AAE?$AAT?$AA?$AN?$AA?6@ 10001320     pwm_mx25_topaz_v1:pwmmdd.obj
 0001:00000368       ??_C@_1GK@CAEOOHBG@?$AAP?$AAW?$AAM?$AA_?$AAD?$AAl?$AAl?$AAE?$AAn?$AAt?$AAr?$AAy?$AA?3?$AA?5?$AAD?$AAL?$AAL?$AA_?$AAP?$AAR?$AAO?$AAC?$AAE?$AAS?$AAS?$AA_?$AAD?$AAE?$AAT?$AAA?$AAC?$AAH@ 10001368     pwm_mx25_topaz_v1:pwmmdd.obj
 0001:000003d8       ??_C@_1GK@GEMLMLOA@?$AAP?$AAW?$AAM?$AA_?$AAD?$AAl?$AAl?$AAE?$AAn?$AAt?$AAr?$AAy?$AA?3?$AA?5?$AAD?$AAL?$AAL?$AA_?$AAP?$AAR?$AAO?$AAC?$AAE?$AAS?$AAS?$AA_?$AAA?$AAT?$AAT?$AAA?$AAC?$AAH@ 100013d8     pwm_mx25_topaz_v1:pwmmdd.obj
 0001:00000444       ??_C@_1BK@HCOBBPHJ@?$AA?9?$AA?9?$AAP?$AAw?$AAm?$AAS?$AAt?$AAa?$AAr?$AAt?$AA?$AN?$AA?6?$AA?$AA@ 10001444     pwm_mx25_topaz_v1:pwmpdd.obj
 0001:00000460       ??_C@_1BK@PNACJAJI@?$AA?$CL?$AA?$CL?$AAP?$AAw?$AAm?$AAS?$AAt?$AAa?$AAr?$AAt?$AA?$AN?$AA?6?$AA?$AA@ 10001460     pwm_mx25_topaz_v1:pwmpdd.obj
 0001:0000047c       ??_C@_1BI@MFJHMLL@?$AA?9?$AA?9?$AAP?$AAw?$AAm?$AAS?$AAt?$AAo?$AAp?$AA?$AN?$AA?6?$AA?$AA@ 1000147c     pwm_mx25_topaz_v1:pwmpdd.obj
 0001:00000494       ??_C@_1BI@MOJFHEGL@?$AA?$CL?$AA?$CL?$AAP?$AAw?$AAm?$AAS?$AAt?$AAo?$AAp?$AA?$AN?$AA?6?$AA?$AA@ 10001494     pwm_mx25_topaz_v1:pwmpdd.obj
 0001:000004ac       ??_C@_1CE@EPEJADJB@?$AA?9?$AA?9?$AAP?$AAw?$AAm?$AAP?$AAl?$AAa?$AAy?$AAS?$AAa?$AAm?$AAp?$AAl?$AAe?$AA?$AN?$AA?6?$AA?$AA@ 100014ac     pwm_mx25_topaz_v1:pwmpdd.obj
 0001:000004d0       ??_C@_1CE@FNIEBCNJ@?$AA?$CL?$AA?$CL?$AAP?$AAw?$AAm?$AAP?$AAl?$AAa?$AAy?$AAS?$AAa?$AAm?$AAp?$AAl?$AAe?$AA?$AN?$AA?6?$AA?$AA@ 100014d0     pwm_mx25_topaz_v1:pwmpdd.obj
 0001:000004f4       ??_C@_1BO@PAFDLCMG@?$AA?9?$AA?9?$AAP?$AAw?$AAm?$AAR?$AAe?$AAl?$AAe?$AAa?$AAs?$AAe?$AA?$AN?$AA?6?$AA?$AA@ 100014f4     pwm_mx25_topaz_v1:pwmpdd.obj
 0001:00000514       ??_C@_1BO@HMKNPGLI@?$AA?$CL?$AA?$CL?$AAP?$AAw?$AAm?$AAR?$AAe?$AAl?$AAe?$AAa?$AAs?$AAe?$AA?$AN?$AA?6?$AA?$AA@ 10001514     pwm_mx25_topaz_v1:pwmpdd.obj
 0001:00000534       ??_C@_1CE@MGGINJHD@?$AA?9?$AA?9?$AAP?$AAw?$AAm?$AAI?$AAn?$AAi?$AAt?$AAi?$AAa?$AAl?$AAi?$AAz?$AAe?$AA?$AN?$AA?6?$AA?$AA@ 10001534     pwm_mx25_topaz_v1:pwmpdd.obj
 0001:00000558       ??_C@_1EO@NJNKCGCL@?$AAP?$AAw?$AAm?$AAI?$AAn?$AAi?$AAt?$AAi?$AAa?$AAl?$AAi?$AAz?$AAe?$AA?3?$AA?5?$AA?5?$AAM?$AAm?$AAM?$AAa?$AAp?$AAI?$AAo?$AAS?$AAp?$AAa?$AAc?$AAe?$AA?5?$AAf?$AAa?$AAi@ 10001558     pwm_mx25_topaz_v1:pwmpdd.obj
 0001:000005a8       ??_C@_1FE@IDHDOEDF@?$AAP?$AAw?$AAm?$AAI?$AAn?$AAi?$AAt?$AAi?$AAa?$AAl?$AAi?$AAz?$AAe?$AA?3?$AA?5?$AA?5?$AAC?$AAo?$AAu?$AAl?$AAd?$AA?5?$AAn?$AAo?$AAt?$AA?5?$AAr?$AAe?$AAa?$AAd?$AA?5?$AAr@ 100015a8     pwm_mx25_topaz_v1:pwmpdd.obj
 0001:000005fc       ??_C@_1CE@NEKFMIDL@?$AA?$CL?$AA?$CL?$AAP?$AAw?$AAm?$AAI?$AAn?$AAi?$AAt?$AAi?$AAa?$AAl?$AAi?$AAz?$AAe?$AA?$AN?$AA?6?$AA?$AA@ 100015fc     pwm_mx25_topaz_v1:pwmpdd.obj
 0001:00000620       ??_C@_1BK@CGFLKAA@?$AA?9?$AA?9?$AAP?$AAw?$AAm?$AAR?$AAe?$AAs?$AAe?$AAt?$AA?$AN?$AA?6?$AA?$AA@ 10001620     pwm_mx25_topaz_v1:pwmpdd.obj
 0001:0000063c       ??_C@_1BK@INIGDFOB@?$AA?$CL?$AA?$CL?$AAP?$AAw?$AAm?$AAR?$AAe?$AAs?$AAe?$AAt?$AA?$AN?$AA?6?$AA?$AA@ 1000163c     pwm_mx25_topaz_v1:pwmpdd.obj
 0001:00000658       ??_C@_1CI@EINNJFIP@?$AA?9?$AA?9?$AAP?$AAw?$AAm?$AAR?$AAe?$AAa?$AAd?$AAR?$AAe?$AAg?$AAi?$AAs?$AAt?$AAe?$AAr?$AA?$AN?$AA?6?$AA?$AA@ 10001658     pwm_mx25_topaz_v1:pwmpdd.obj
 0001:00000680       ??_C@_1CI@IGHEPEFB@?$AA?$CL?$AA?$CL?$AAP?$AAw?$AAm?$AAR?$AAe?$AAa?$AAd?$AAR?$AAe?$AAg?$AAi?$AAs?$AAt?$AAe?$AAr?$AA?$AN?$AA?6?$AA?$AA@ 10001680     pwm_mx25_topaz_v1:pwmpdd.obj
 0001:000006a8       ??_C@_1KA@HPHHJN@?$AAP?$AAw?$AAm?$AAG?$AAe?$AAt?$AAR?$AAe?$AAg?$AAi?$AAs?$AAt?$AAr?$AAy?$AAV?$AAa?$AAl?$AAu?$AAe?$AAs?$AA?3?$AA?5?$AAE?$AAr?$AAr?$AAo?$AAr?$AA?0?$AA?5?$AAc?$AAa?$AAn@ 100016a8     pwm_mx25_topaz_v1:pwmpdd.obj
 0001:00000748       ??_C@_1M@EENNDIOJ@?$AAI?$AAn?$AAd?$AAe?$AAx?$AA?$AA@ 10001748     pwm_mx25_topaz_v1:pwmpdd.obj
 0001:00000758       ??_C@_1IC@OLBJJLPP@?$AAP?$AAw?$AAm?$AAG?$AAe?$AAt?$AAR?$AAe?$AAg?$AAi?$AAs?$AAt?$AAr?$AAy?$AAV?$AAa?$AAl?$AAu?$AAe?$AAs?$AA?3?$AA?5?$AAE?$AAr?$AAr?$AAo?$AAr?$AA?5?$AAc?$AAa?$AAn?$AA?5@ 10001758     pwm_mx25_topaz_v1:pwmpdd.obj
 0001:000007dc       ??_C@_1CI@OHCJFJPM@?$AAE?$AAR?$AAR?$AAO?$AAR?$AA?3?$AA?5?$AA?$CF?$AAs?$AA?5?$AAl?$AAi?$AAn?$AAe?$AA?5?$AA?$CF?$AAd?$AA?3?$AA?5?$AA?$AA@ 100017dc     pwm_mx25_topaz_v1:pwmpdd.obj
 0001:00000808       ??_C@_1KA@KPOCIOPJ@?$AAc?$AA?3?$AA?2?$AAw?$AAi?$AAn?$AAc?$AAe?$AAr?$AAo?$AAo?$AAt?$AAs?$AA?2?$AAt?$AAo?$AAp?$AAa?$AAz?$AA?2?$AAw?$AAi?$AAn?$AAc?$AAe?$AA7?$AA0?$AA0?$AA?2?$AAp?$AAl?$AAa@ 10001808     pwm_mx25_topaz_v1:pwmpdd.obj
 0001:000008c8       BSPGetPWMClockSource       100018c8 f   bsppwm.obj
 0001:000008e0       BSPPwmSetClockGatingMode   100018e0 f   bsppwm.obj
 0001:000009cc       BSPPwmIomuxSetPin          100019cc f   bsppwm.obj
 0001:00000a94       BSPPwmGetBaseAddress       10001a94 f   bsppwm.obj
 0001:00000b4c       PWM_Init                   10001b4c f   pwm_mx25_topaz_v1:pwmmdd.obj
 0001:00000bb0       PWM_Deinit                 10001bb0 f   pwm_mx25_topaz_v1:pwmmdd.obj
 0001:00000c40       PWM_Open                   10001c40 f   pwm_mx25_topaz_v1:pwmmdd.obj
 0001:00000e34       PWM_Close                  10001e34 f   pwm_mx25_topaz_v1:pwmmdd.obj
 0001:0000101c       PWM_PowerDown              1000201c f   pwm_mx25_topaz_v1:pwmmdd.obj
 0001:00001098       PWM_PowerUp                10002098 f   pwm_mx25_topaz_v1:pwmmdd.obj
 0001:0000111c       PWM_Read                   1000211c f   pwm_mx25_topaz_v1:pwmmdd.obj
 0001:000011d8       PWM_Write                  100021d8 f   pwm_mx25_topaz_v1:pwmmdd.obj
 0001:000012a8       PWM_IOControl              100022a8 f   pwm_mx25_topaz_v1:pwmmdd.obj
 0001:00001670       PWM_DllEntry               10002670 f   pwm_mx25_topaz_v1:pwmmdd.obj
 0001:0000173c       PwmStart                   1000273c f   pwm_mx25_topaz_v1:pwmpdd.obj
 0001:000017e4       PwmStop                    100027e4 f   pwm_mx25_topaz_v1:pwmpdd.obj
 0001:00001888       PwmPlaySample              10002888 f   pwm_mx25_topaz_v1:pwmpdd.obj
 0001:00001b34       PwmDeinit                  10002b34 f   pwm_mx25_topaz_v1:pwmpdd.obj
 0001:00001c04       PwmInitialize              10002c04 f   pwm_mx25_topaz_v1:pwmpdd.obj
 0001:00001dbc       PwmReset                   10002dbc f   pwm_mx25_topaz_v1:pwmpdd.obj
 0001:00001e60       PwmReadRegister            10002e60 f   pwm_mx25_topaz_v1:pwmpdd.obj
 0001:00002104       SetPwmPower                10003104 f   pwm_mx25_topaz_v1:pwmpdd.obj
 0001:000021a0       PwmGetRegistryValues       100031a0 f   pwm_mx25_topaz_v1:pwmpdd.obj
 0001:000022a4       PwmOpen                    100032a4 f   pwm_mx25_topaz_v1:pwmpdd.obj
 0001:000022d4       NKDbgPrintfW               100032d4 f   coredll:COREDLL.dll
 0001:000022e4       LocalAlloc                 100032e4 f   coredll:COREDLL.dll
 0001:000022f4       LocalFree                  100032f4 f   coredll:COREDLL.dll
 0001:00002304       SetLastError               10003304 f   coredll:COREDLL.dll
 0001:00002314       DisableThreadLibraryCalls  10003314 f   coredll:COREDLL.dll
 0001:00002324       RegisterDbgZones           10003324 f   coredll:COREDLL.dll
 0001:00002334       GetTickCount               10003334 f   coredll:COREDLL.dll
 0001:00002344       LeaveCriticalSection       10003344 f   coredll:COREDLL.dll
 0001:00002354       EnterCriticalSection       10003354 f   coredll:COREDLL.dll
 0001:00002364       DeleteCriticalSection      10003364 f   coredll:COREDLL.dll
 0001:00002374       InitializeCriticalSection  10003374 f   coredll:COREDLL.dll
 0001:00002384       RegQueryValueExW           10003384 f   coredll:COREDLL.dll
 0001:00002394       GetLastError               10003394 f   coredll:COREDLL.dll
 0001:000023a4       OpenDeviceKey              100033a4 f   coredll:COREDLL.dll
 0001:000023b4       MmUnmapIoSpace             100033b4 f   ceddk:CEDDK.dll
 0001:000023c4       MmMapIoSpace               100033c4 f   ceddk:CEDDK.dll
 0001:000023d4       DDKClockSetGatingMode      100033d4 f   cspddk:CSPDDK.dll
 0001:000023e4       DDKIomuxSetPinMux          100033e4 f   cspddk:CSPDDK.dll
 0001:000023f4       DDKClockGetFreq            100033f4 f   cspddk:CSPDDK.dll
 0001:00002404       __security_init_cookie     10003404 f   corelib0:seccinit.obj
 0001:0000249c       __GSHandlerCheck           1000349c f   corelib0:gshandler.obj
 0001:000024e0       __GSHandlerCheckCommon     100034e0 f   corelib0:gshandler.obj
 0001:00002584       __security_check_cookie    10003584 f   corelib0:armsecgs.obj
 0001:00002594       __gsfailure                10003594     corelib0:armsecgs.obj
 0001:000025d8       memset                     100035d8 f   corelib1:COREDLL.dll
 0001:000025e8       memcpy                     100035e8 f   corelib1:COREDLL.dll
 0001:000025f8       __rt_udiv                  100035f8 f   corelib1:COREDLL.dll
 0001:00002608       __security_gen_cookie2     10003608 f   corelib1:COREDLL.dll
 0001:00002618       __report_gsfailure         10003618 f   corelib1:COREDLL.dll
 0001:0000262c       __IMPORT_DESCRIPTOR_COREDLL 1000362c     coredll:COREDLL.dll
 0001:00002640       __IMPORT_DESCRIPTOR_CEDDK  10003640     ceddk:CEDDK.dll
 0001:00002654       __IMPORT_DESCRIPTOR_CSPDDK 10003654     cspddk:CSPDDK.dll
 0001:00002668       __NULL_IMPORT_DESCRIPTOR   10003668     coredll:COREDLL.dll
 0002:00000000       __imp_MmUnmapIoSpace       10004000     ceddk:CEDDK.dll
 0002:00000004       __imp_MmMapIoSpace         10004004     ceddk:CEDDK.dll
 0002:00000008       \177CEDDK_NULL_THUNK_DATA  10004008     ceddk:CEDDK.dll
 0002:0000000c       __imp_SetLastError         1000400c     coredll:COREDLL.dll
 0002:00000010       __imp_DisableThreadLibraryCalls 10004010     coredll:COREDLL.dll
 0002:00000014       __imp_RegisterDbgZones     10004014     coredll:COREDLL.dll
 0002:00000018       __imp_GetTickCount         10004018     coredll:COREDLL.dll
 0002:0000001c       __imp_LeaveCriticalSection 1000401c     coredll:COREDLL.dll
 0002:00000020       __imp_LocalFree            10004020     coredll:COREDLL.dll
 0002:00000024       __imp_DeleteCriticalSection 10004024     coredll:COREDLL.dll
 0002:00000028       __imp_InitializeCriticalSection 10004028     coredll:COREDLL.dll
 0002:0000002c       __imp_RegQueryValueExW     1000402c     coredll:COREDLL.dll
 0002:00000030       __imp_GetLastError         10004030     coredll:COREDLL.dll
 0002:00000034       __imp_OpenDeviceKey        10004034     coredll:COREDLL.dll
 0002:00000038       __imp_LocalAlloc           10004038     coredll:COREDLL.dll
 0002:0000003c       __imp_EnterCriticalSection 1000403c     coredll:COREDLL.dll
 0002:00000040       __imp_NKDbgPrintfW         10004040     coredll:COREDLL.dll
 0002:00000044       __imp___security_gen_cookie2 10004044     corelib1:COREDLL.dll
 0002:00000048       __imp___rt_udiv            10004048     corelib1:COREDLL.dll
 0002:0000004c       __imp_memcpy               1000404c     corelib1:COREDLL.dll
 0002:00000050       __imp_memset               10004050     corelib1:COREDLL.dll
 0002:00000054       __imp___report_gsfailure   10004054     corelib1:COREDLL.dll
 0002:00000058       \177COREDLL_NULL_THUNK_DATA 10004058     coredll:COREDLL.dll
 0002:0000005c       __imp_DDKIomuxSetPinMux    1000405c     cspddk:CSPDDK.dll
 0002:00000060       __imp_DDKClockSetGatingMode 10004060     cspddk:CSPDDK.dll
 0002:00000064       __imp_DDKClockGetFreq      10004064     cspddk:CSPDDK.dll
 0002:00000068       \177CSPDDK_NULL_THUNK_DATA 10004068     cspddk:CSPDDK.dll
 0002:00000070       dpCurSettings              10004070     pwm_mx25_topaz_v1:pwmmdd.obj
 0002:000004b4       __security_cookie          100044b4     corelib0:seccinit.obj
 0002:000004b8       __security_cookie_complement 100044b8     corelib0:seccinit.obj

 entry point at        0001:00001670

 Static symbols

 0001:00001fc0       Reset                      10002fc0 f   pwm_mx25_topaz_v1:pwmpdd.obj
 0001:00002098       PWMSetPrescalerDiv         10003098 f   pwm_mx25_topaz_v1:pwmpdd.obj
